:100000000C94EC060C9414070C9414070C9414072D
:100010000C9414070C9414070C9414070C941407F4
:100020000C9414070C9414070C9414070C94E331EB
:100030000C9414070C9414070C9414070C941407D4
:100040000C9456320C9414070C9414070C94140757
:100050000C9414070C9414070C9414070C941407B4
:100060000C941D220C94140705A84CCDB2D44EB9A3
:100070003836A9020C50B9918688083CA6AAAA2A4B
:10008000BE000000803F50726573732041006174B0
:1000900020747261636B20002E20506C61636500D8
:1000A000596F7520726561636865642000436F6EE7
:1000B00067726174756C6174696F6E73212000548E
:1000C0007261636B206C6F636B6564002F00204C62
:1000D0003A0020506F733A005370643A004C454622
:1000E000540052494748540063757272656E74201B
:1000F0004469723A200070726573732043207768F8
:10010000656E20646F6E65007475726E207269672B
:1001100068742B7072657373205249474854007499
:1001200075726E206C6566742B7072657373204CEB
:10013000454654004144584C3334352063616C6962
:1001400062726174696F6E001573656C656374200B
:1001500016636C65617220176261636B002D2D3A26
:100160002D2D202D2D00200030003A0030002000E1
:10017000100020547261636B202020202020205426
:10018000696D6520506F7300636F756C64206E6FCE
:1001900074206F70656E204441542066696C650060
:1001A000422D52616C6C79000002FA01F201EA0101
:1001B000E401DE01D601CE01C501BC0148617264D3
:1001C000657374320048617264657374310048610C
:1001D0007264657232004861726465723100486110
:1001E000726432004861726431004D656469756DF6
:1001F00032004D656469756D310045617379320077
:1002000045617379310042023A022D022802180238
:1002100042023A022D02280243616C6962726174E3
:100220006520416363656C00457869740053656CB3
:1002300065637420747261636B00526573746172DC
:100240007400526573756D65001010FFFF800187A3
:10025000E187F18071807183E183E1807180718039
:100260007187F187C180018001FFFF1010FFFF80BF
:100270000187C187E184E180E181E183E187C18772
:10028000818E018FE18FE180018001FFFF1010FF5F
:10029000FF800180C187C187C185C181C181C181C2
:1002A000C181C181C181C181C180018001FFFF1075
:1002B0001000003C1E3C3C3C3C1E3C1E381E780E90
:1002C000780F700F7007F007E007E007E003C00049
:1002D00000101000001FE01FF81FF81E7C1E781E83
:1002E000781FF01FE01FF01EF81E781E781E7C1E7F
:1002F0003C00001010000007E00FF81FFC3E7C3CA3
:100300003C3C3E7C1E7C1E3C3E3C3C3FFC1FF80FB0
:10031000F003C0000010100000FC3FFC3FFE3FEE69
:100320003FEE7FEE7FEF7FEF6FE7EFE7EFE7EFE77F
:10033000CFE3CFE3CF00001010000003F80FF81F49
:10034000F83F083E003C003CFC3CFC3CFC3E3C3F93
:100350003C1FFC0FFC03F00000101000000FF00F1A
:10036000F00FF00FF00F000F000FF00FF00FF00F75
:10037000000F000FF80FF80FF80000101000000336
:10038000E007E007E007F00FF00F700E781E781F0F
:10039000F81FFC3FFC3C3C3C3E7C1E000000010280
:1003A00003040505060607070808090909090A0ADA
:1003B0000A0A0A0A0A0A0B0B0B0B0B0B0B0B0C0C91
:1003C0000C0C0C0C0C0C0D0D0D0D0D0D0D0D0E0E61
:1003D0000E0E0E0E0E0E0F0F0F0F0F0F0F0F090642
:1003E0000D01080F01050B0F0104090C0F00030597
:1003F000070B0E0F01030507090B0D0F0001030585
:1004000007090B0D0F0002030506080A0C0D0F006B
:100410000103040607090B0C0E0F00010304050776
:1004200008090B0C0E0F00010204050607080A0B51
:100430000D0E0F0001020304060708090A0C0D0E39
:100440000F0001020304050607090A0B0C0D0E0F2D
:10045000000102030405060708090A0B0C0D0E0F24
:100460001010F0F0F0F0F0F0F0F00F0F0F0F0F0F92
:100470000F0FF0F0F0F0F0F0F0F00F0F0F0F0F0F84
:100480000F0F10107FFEFFFFE007C663C663C66351
:10049000C663CE73CC33D81BD81BD81BC003E00770
:1004A000FFFF7FFE10107FFEFFFFC007CC03CF03CE
:1004B000C3C3C0F3C03BC03BC0F3C3C3CF03CC0333
:1004C000E007FFFF7FFE10107FFEFFFFE007C03355
:1004D000C0F3C3C3CF03DC03DC03CF03C3C3C0F348
:1004E000C033E003FFFF7FFEFFC000FFE000FFE03E
:1004F00000FFF000FFF000FFF800FFF800FFFC0035
:10050000FFFC00FFFE00FFFE00FFFF00FFFFC0FF3B
:10051000FE70FFFE18FFFE18FFFE0CFFFE30FFFC12
:10052000C0FFFCC0FFFD80FFF300FFEC00FFEC000C
:10053000FFB800FE6000FDC000FDC000FB0000F73A
:100540008000EF8000EF8000FFC000FFC000FFE0F0
:1005500000FFE000FFE000FFF000FFE800FFE40024
:10056000FFE400FFC400FFD800FFB000FFB000FFB1
:100570006000FEC000FD8000FD8000F30000E6008A
:1005800000EF0000EF0000FF8000FF8000FFC000D0
:10059000FFC000FFC000FFE000FFF000FFF000FF21
:1005A000F000FFF800FFFC00FFFE00FFFE00FFFD73
:1005B00080FFFC40FFF860FFF860FFC180FE3E0056
:1005C000FFE000FFE000FFC000FFE000FFF000FFE1
:1005D000D800FFD800FFB000FF6000FEC000FF8021
:1005E00000FF0000FE0000FC0000F80000F8000022
:1005F000F80000F80000FF0000FD0000FF8000FF91
:100600008020F800A0FE0020FE0040F80060FC0002
:1006100010FC00A0FFE040FEA020FFC040FC00A8AE
:10062000FFA000FC1010FFC000FFC400F80000FF96
:10063000F280FAB040FFC080FFC040F800C0FF0069
:1006400020FD0080FF0040F80080FC0020FC0080BE
:10065000FE0160FE0000FE0000FE0000FF0000FF43
:100660008000FFC000FFC000101001C00220022067
:1006700001E00020022001C000000FF0B81D700E44
:10068000FFFFFFFFFFFF781E700E101003C0042055
:10069000042003C00420042003C000000FF0B81D94
:1006A000700EFFFFFFFFFFFF781E700E101003C0DB
:1006B00000400040008001000100010000000FF038
:1006C000B81D700EFFFFFFFFFFFF781E700E1010A9
:1006D00001800240020003800240024001800000CD
:1006E0000FF0B81D700EFFFFFFFFFFFF781E700EAA
:1006F000101003C00200038000400040024001804F
:1007000000000FF0B81D700EFFFFFFFFFFFF781E07
:10071000700E10100080010001000200028003C072
:10072000008000000FF0B81D700EFFFFFFFFFFFFFD
:10073000781E700E101001800240004000800040C2
:100740000240018000000FF0B81D700EFFFFFFFF98
:10075000FFFF781E700E10100180024000400080E4
:100760000100020003C000000FF0B81D700EFFFF73
:10077000FFFFFFFF781E700E1010026006900A90B7
:10078000029002900290026000000FF0B81D700EFF
:10079000FFFFFFFFFFFF781E700E1010008001802A
:1007A0000280008000800080008000000FF0B81DF3
:1007B000700EFFFFFFFFFFFF781E700EFFFFFFFFB1
:1007C000F3FFC00FC003C0018001800180018001E0
:1007D0008001800000000000000000000000000117
:1007E00000018001F803FC0FFFFFFFFF0000000085
:1007F000040032F030BC3A3C743E7A3C743E693EB0
:10080000743E603EE43DE0BEC0BDE0FDC0F9C0E620
:10081000F11E7EBE055C02B000000000000000007A
:10082000080031F03AB8303C7A3C743E6A3C753E80
:10083000683E643FE03EE8BDE0BDC0FDC0F9E04673
:10084000F0BE7D5E04BC035000000000FFFFFFFF10
:10085000FC0FF8038001000100010000000000000F
:100860000000000080008001800180018001800183
:10087000C001C003C00FF3FFFFFFFFFF0000000037
:1008800002B0055C7EBEF11EC0E6C0F9E0FDC0BD51
:10089000E0BEE43D603E743E693E743E7A3C743E88
:1008A0003A3C30BC32F004000000000000000000C0
:1008B000035004BC7D5EF0BEE046C0F9C0FDE0BD63
:1008C000E8BDE03E643F683E753E6A3C743E7A3C5B
:1008D000303C3AB831F0080000000000FFFFFBFF99
:1008E000E00FC003C003C0018001800180018001CE
:1008F0000000000000000000000000008001F00186
:10090000F801FC01FE03FE07FF9FFFFF000004004B
:1009100018B03A383878367E7C7E6C7C607C4178C2
:10092000C179C1F9C1F1C1E1C25DF8BD7D7C0ABEEA
:10093000057E03BE01DC01E8006000000000040049
:1009400018B03A38343C3C7E747E687C6478417CD4
:10095000C179C1F9C1F1C1E3E02DF95D7EBC0D7E25
:1009600006BE035E01FC01F800600000FFFFFF9F70
:10097000FE07FE03FC01F801F00180010000000009
:100980000000000000000000800180018001800163
:10099000C001C003C003E00FFBFFFFFF00000060C9
:1009A00001E801DC03BE057E0ABE7D7CF8BDC25DA8
:1009B000C1E1C1F1C1F9C1794178607C6C7C7C7E78
:1009C000367E38783A3818B0040000000000006025
:1009D00001F801FC035E06BE0D7E7EBCF95DE02DD4
:1009E000C1E3C1F1C1F9C179417C6478687C747E4E
:1009F0003C7E343C3A3818B004000000FFFFFFFF93
:100A0000E3FF003F000F00030001000000000000B2
:100A100000000000000000000000000000010003D2
:100A2000000F003FE3FFFFFFFFFFFFFF000000009C
:100A30001C00F5C0E1B0D5F8E27EDC7CD87DCC7C32
:100A4000D87DDA7CC8FDD87CD8FDC87CC07EC1F8D2
:100A5000C1B0E1C01C000000000000000000000068
:100A60001C00EBC0D1F0C37CD57CE87DDC7CD87D5C
:100A7000D87CCAFDC07CDCFDC87CD0FDC17CC97CB3
:100A8000C1F0E1C01C0000000000000003053F2190
:100A90003F1208120A100A0E1C0E0C1E0C141A1417
:100AA000161F161E131E1E1B1E1E1F1E3F213F3A21
:100AB0002F3A173D173F213F181F02040A041F0E4B
:100AC00004040E1F0A1F0A0E0E1F04110E2E252EDF
:100AD0002F2A2E262929021F02081F08150E04049A
:100AE0000E150E15151B151B040604040C0400003E
:100AF000000017000300031F0A1F16371A190413FA
:100B00000A153A000300000E11110E000A040A042F
:100B10000E040030000404040010001804031F1128
:100B20001F121F101D151711151F07041F17151D64
:100B30001F151D01011F1F151F17151F000A00009B
:100B40003200040A110A0A0A110A040115020E11E0
:100B5000171E051E1F150A0E110A1F110E1F151153
:100B60001F05010E111D1F041F111F1108100F1F5B
:100B7000041B1F10101F061F1E040F0E110E1F094D
:100B8000060E112E1F051A121509011F011F101F35
:100B90000F180F1F0C1F1B041B031C031915130038
:100BA0001F11030418111F00020102202020000160
:100BB000020C121E1F120C0C12120C121F0C1A1413
:100BC000041E05242A1E1F021C141D1020201D1F98
:100BD0000814111F101E041E1E021C0C120C3E0ACB
:100BE000040C123E1E040214160A020F120E101EEE
:100BF0000E100E1E081E120C1226281E322A260463
:100C00001E21001F00211E040102013F213F0A4E48
:100C10006F2053442063617264206F720A6E6F20EC
:100C20004C4F414445522E4845580A0A153A4578DA
:100C30006974001D20466C617368696E670A202024
:100C40006C6F616465722E2E2E0A0A444F4E275433
:100C5000205455524E204F464621000A0A153A4963
:100C6000676E6F7265006D560A0A504C45415345D8
:100C7000205455524E204F464620004C4F5720429C
:100C800041545445525921200017534400161378FB
:100C900000161314001510200015201000540A032C
:100CA000E181867F3E186D830F0F0E0183866033CE
:100CB000186DC3198F1803C38E6033186DE330CFDE
:100CC0001803C39E603630CDE360CF3006C79E7EEA
:100CD0003E30CDB360CF300CC6F6603330D9B6604D
:100CE000CF33CFCCF66061B0DB1E60CF30D86CE67E
:100CF000C061B0DB1E618F19986CC6C063B19B0EDA
:100D0000330F0FB078C6FF7E1F1B061E0F0500892C
:100D10003008023802497868140000F6E8DBCFC3D7
:100D2000B8AEA49B928A827B746E68625C57524E06
:100D30004945413E3A3734312E2C29272523211F9E
:100D40001D1C1A1917161514131211100F0E0D0C65
:100D50000B0A090807064500680100000500680144
:100D6000380100000500380168010000740D700DA5
:100D70000101FF030101F703000000080002010068
:100D80000003040700000000000000000102040846
:100D900010204080010204081020010204081020E5
:100DA0000404040404040404020202020202030311
:100DB00003030303000000002300260029000000B5
:100DC0000000250028002B00000000002400270060
:100DD0002A002C11D21F332111241FBECFEFD8E0DF
:100DE000DEBFCDBF11E0A0E0B1E0E4E8F5E702C06E
:100DF00005900D92A23DB107D9F728E0A2EDB1E030
:100E000001C01D92A432B207E1F71DE0C8EDDDE09C
:100E100004C02297FE010E944E39C23DD107C9F796
:100E20000E942D360C94C03A0C9400008FEF8EBDBA
:100E30000DB407FEFDCF8EB508958EBD0DB407FE2F
:100E4000FDCF08950C94AA3A0C94B23ADC016435B3
:100E500008F053C0403308F050C090968C919097A2
:100E6000342F359535953595E62FFF27E7FDF0951D
:100E7000242F2770823099F4DF01A05FB94F84E5F9
:100E80003802A00DB11D11248C9190E0022E02C0F9
:100E9000959587950A94E2F78095817009C0833013
:100EA00039F446271C968C91482740FF03C014C094
:100EB000811112C084E53802E00DF11D1124E05FBC
:100EC000F94F81E090E0022E01C0880F0A94EAF702
:100ED00080959081982310C084E53802E00DF11DC3
:100EE0001124E05FF94F81E090E0022E01C0880FED
:100EF0000A94EAF79081982B90830895CF92DF921D
:100F0000EF92FF926B017C012DE137E046E157E063
:100F10006AE070E088E195E00E94A61F83E891E016
:100F20000E94DD1C892B41F4C701B601FF90EF90B0
:100F3000DF90CF900C942C1E48EC68E871E08FE7AE
:100F400094E0FF90EF90DF90CF900C94CE29CF9358
:100F5000DF9300D000D000D0CDB7DEB745EF51E031
:100F600064E070E087EF91E00E942C1D9093F40103
:100F70008093F301892B51F16091DA0170E080E0F8
:100F800090E021E1660F771F881F991F2A95D1F7FE
:100F90002091EA013091EB01220F331F220F331F02
:100FA000620F731F811D911D6C5F7F4F8F4F9F4F8D
:100FB0000E947E0745EF51E064E070E087EF91E02A
:100FC0000E942C1D9093F4018093F3013091F8015D
:100FD0005091F9015F5F6091FA012091F70140E0C3
:100FE00070E080E090E026960FB6F894DEBF0FBE6A
:100FF000CDBFDF91CF91089563E570E080E595E086
:101000000E94B72080E595E00E943021811103C045
:1010100081E08093D7010895CF93DF9362EB80E066
:1010200090E00E9424076CEA81E090E00E9424078F
:1010300062EE82E090E00E942407C3E0D0E0CE019F
:101040000E942207882321F060E0CE010E9424073D
:101050002196C11584E0D80791F7DF91CF910895CB
:1010600080E090E00E942207823B61F481E090E002
:101070000E9422078C3A31F482E090E00E9422071D
:10108000823E39F00E940C081092DA0110920F0192
:10109000089584E090E00E9422078093DA0185E0C1
:1010A00090E00E94220780930F0108958F929F92F3
:1010B000AF92BF92CF92DF92EF92FF920F931F9366
:1010C000CF93DF93982E862EEA0180E090E00E9475
:1010D0002207823B61F481E090E00E9422078C3A73
:1010E00031F482E090E00E942207823E71F0DF91AD
:1010F000CF911F910F91FF90EF90DF90CF90BF9015
:10110000AF909F908F900C940C08CE0164E170E03A
:101110000E94C938EB01A92CB12C7501EE0CFF1C03
:10112000EE0CFF1C670136E0C30ED11CC6010E9405
:1011300022078701095F1F4F9701285F3F4F790101
:101140008823B9F0881620F4682DC6010E94240770
:10115000C8010E942207D82EC7010E9422072D2D08
:1011600030E0322F2227280F311DC217D30768F431
:1011700004C0682DC6010E9424076D2FC8010E947B
:1011800024076C2FC7010E9424079092D90123E005
:10119000281598F020910E0130E021503109A21657
:1011A000B3061CF493949092D9018091D901909147
:1011B0000F01981710F480930F0184E090E00E94D3
:1011C00022076091D901861721F084E090E00E9407
:1011D000240785E090E00E94220760910F018617A6
:1011E00081F085E090E0DF91CF911F910F91FF900A
:1011F000EF90DF90CF90BF90AF909F908F900C9426
:101200002407DF91CF911F910F91FF90EF90DF9016
:10121000CF90BF90AF909F908F9008950F931F93A2
:10122000413308F08FC0853591050CF08BC077FDF8
:1012300089C0342F3770E1E0F0E001C0EE0F3A953D
:10124000EAF75E2FAE2FA095E42FE695E695E6959A
:1012500034E5E39FF001112497FF02C080E090E0A5
:101260008E0F9F1F6535710514F064E570E06E0FF9
:101270007F1F21110FC0861797070CF063C0E09104
:101280007D04F0917E04E80FF91F20812A2320833A
:101290000196F1CF213079F4861797070CF052C0F0
:1012A000E0917D04F0917E04E80FF91F2081252B49
:1012B00020830196F1CF233009F044C00091F0045F
:1012C0001091F1042091F2043091F304040F111DE8
:1012D000211D311D6150710900FF1AC08617970743
:1012E0008CF5E0917D04F0917E04E80FF91F2081D8
:1012F000252B208302969C0121503109E0917D0429
:10130000F0917E04E20FF31F20812A232083E6CF91
:1013100086179707BCF4E0917D04F0917E04E80FF6
:10132000F91F20812A23208302969C012150310934
:10133000E0917D04F0917E04E20FF31F2081252BC4
:101340002083E6CF1F910F9108952F923F924F92E5
:101350005F926F927F928F929F92AF92BF92CF9245
:10136000DF92EF92FF920F931F93CF93DF9300D002
:101370001F92CDB7DEB741504F3008F090C0853591
:1013800008F08DC0613308F08AC0480152E0850E34
:10139000911C30E050E00FE010E03801641A750A4B
:1013A0005A01AA0CBB1CA501475D5E4F5B834A83B3
:1013B000262E312C90E0EE24E394F12C632F70E084
:1013C000661577050CF06BC0EA81FB81C080D18087
:1013D000F601E60FF71F4491F401E40FF11DE40F4D
:1013E000F11DB4903196A490DB01A20DB31DAD01A7
:1013F000F3E055954795FA95E1F7473009F44DC06C
:10140000F4E5F49FB001F59F700D1124680F791F6A
:10141000605F794FA770BB27A70102C0440F551F1B
:10142000AA95E2F7DA0149834B2D50E0542F442767
:101430004A0D511D512C4A2E4094A52DB0E0A61501
:10144000B7055CF5F601EA0FFB1FE4915D01A80EFC
:10145000B91EF4E5AF16B104F4F45801AE1AB108A0
:10146000F501570102C0AA0CBB1CEA95E2F7F50191
:10147000A422B522AE16BF0639F4A60FB71FBC9042
:10148000A980BA28BC9207C0222329F0A60FB71F53
:10149000EC91E421EC935394D0CF3F5F8FCF0F902A
:1014A0000F900F90DF91CF911F910F91FF90EF90D0
:1014B000DF90CF90BF90AF909F908F907F906F9074
:1014C0005F904F903F902F90089520E030E09FEF85
:1014D00087FD805863E08602A0011124FA01E651DD
:1014E000FB4FE491A0917D04B0917E04A20FB31F45
:1014F000EC93FA01E751FB4FE49160917D04709108
:101500007E04620F731FDB01AC5ABF4FEC93FA01EC
:10151000E851FB4F449160917D0470917E04620F0D
:10152000731FFB01E855FF4F408340917D045091AC
:101530007E04420F531FFA01E450FF4F9083409105
:101540007D0450917E04420F531FFA01E05BFE4F71
:1015500090838F5F2F5F3F4F2435310509F0B8CF5F
:101560000895EF92FF920F931F93CF93DF939927E4
:1015700087FD909582599E4FC0917D04D0917E0445
:10158000C80FD91FDE01AC5ABF4F80E090E070E079
:10159000660F771FAB01435A5E4F8B010B581E4FEE
:1015A00067597E4FFA0120813181280F391FF901D7
:1015B00034912C9123232C939C012F5F3F4FFA01F0
:1015C000E080F180E20EF31EF701E490F881FE2145
:1015D000F883E091F004E0FF02C0FB0101C0F801D4
:1015E000E080F180E80EF91EF701E490FC91FE29FD
:1015F000FC93E091F004E0FF02C0FB0101C0F801A0
:10160000E080F180E20EF31EF701E49028812E299C
:101610002993029611968033910509F0C3CFDF918B
:10162000CF911F910F91FF90EF900895CF93E82FE6
:101630008091F00480FD02C0FAEA01C0F5E5CF2FE9
:10164000C09580E390E08E1B9109E7FD939568E0DB
:1016500070E00E94DD38682FE7FDE95FE595E595CC
:10166000E595611101C0E15091E09E0F9630ACF418
:1016700024E59202A0011124405F594F20E030E0A0
:10168000DA01A20FB31FFC931196CC932E5F3F4F4C
:1016900024353105A9F79F5FE9CF662341F147E083
:1016A00050E0481B510987FD539521E030E0042E9E
:1016B00001C0220F0A94EAF721953F2F3223C2235B
:1016C000209584E5E89FF0011124E05FF94FDF01E8
:1016D000119690E080818223832B80838C918223DA
:1016E0008C2B8C939E5F32961296943599F7CF91FE
:1016F00008950F931F93CF93DF93C091F201D6E02B
:10170000CC23A1F08C2F90E00197D89FF001D99FB6
:10171000F00D1124E15AFD4F008111812581438193
:10172000648182810E94A509C150EACFDF91CF91E7
:101730001F910F91089568ED70E08DEC94E00E9488
:10174000BF344AE050E0609111018DEC94E00E94BA
:10175000C13562ED70E08DEC94E00E94BF344AE048
:1017600050E06091DF018DEC94E00E94C1356EEC99
:1017700070E08DEC94E00E94BF348091EA0190917A
:10178000EB018654910960910A0170910B010E944E
:10179000C93877276F5F7F4F4AE050E08DEC94E0C7
:1017A0000E94AC356CEC70E08DEC94E00E94BF348C
:1017B00080910C0190910D0160910A0170910B01D3
:1017C0000E94C9384AE050E08DEC94E00C94C13599
:1017D000EF92FF920F931F93CF93DF938C01EB0156
:1017E000F42EE22E01978E379105A0F461E02613C6
:1017F00060E08DEC94E00E94F0244F2D6FEF600FBD
:101800008DEC94E00E9426074F2D602F8DEC94E024
:101810000E94260760E08DEC94E00E94F0240F37D0
:1018200011052CF5C2388FEFD807D4F461E0E61229
:1018300060E08DEC94E00E94F0244F2D6C2F8DEC35
:1018400094E00E9426076C2F6F5F4F2D8DEC94E083
:10185000DF91CF911F910F91FF90EF900C9426078D
:1018600020E04F2DBE01C80101960E940E09C4352B
:10187000D105E4F2DF91CF911F910F91FF90EF908E
:1018800008950F939091F201953178F456E0959F69
:10189000F0011124E15AFD4F838362834483318335
:1018A000208305839F5F9093F2010F9108957F92AB
:1018B0008F929F92AF92BF92CF92DF92EF92FF9260
:1018C0000F931F93CF93DF931092EB011092EA01D5
:1018D0001092E1011092ED011092EC0110921101B1
:1018E0006091DA0170E080E090E0E1E1660F771F3F
:1018F000881F991FEA95D1F70E942C1E45EF51E0F1
:1019000062E070E087EF91E00E942C1D9093F4015B
:101910008093F3018091F70190E0982F8827209120
:10192000F801820F911D90930D0180930C0145EFFA
:1019300051E062E070E087EF91E00E942C1D9093EF
:10194000F4018093F3018091F70190E0982F8827AC
:101950002091F801820F911D90930B0180930A0151
:1019600000E010E0B6E0FB2EF09EE001F19ED00D0D
:101970001124C952DD4F0E94A707288339834A8367
:101980005B836C837D838091EA019091EB010196EA
:101990009093EB018093EA010F5F1F4F063411050E
:1019A00019F70BEF11E087E4A82E81E0B82E94E040
:1019B000E92E92E0F92E24E5C22E23E0D22ECBE0D0
:1019C000D0E03BE0732E4EE1842E5CE0952E672D37
:1019D0006C1BF801D383C283F501819191915F0162
:1019E000F80191838083F7013597862F8170889D58
:1019F000802D11248F50808370E080E090E00E9461
:101A0000393720E030E040E251E40E94A5369B01E6
:101A1000AC0160E070E080E090E40E943D36F801A7
:101A20006583768387839087F7011082892D8C1BCD
:101A3000F60180832197065F1F4FFAE0EF0EF11C3D
:101A400086E0C81AD108C130D10509F68BE0809331
:101A5000DF011092DE011092DD018CE38093DB0147
:101A600083E08093DC01E091DA01F0E0EE0FFF1FEC
:101A7000E855FE4F659174914CE38FE794E0DF9158
:101A8000CF911F910F91FF90EF90DF90CF90BF907B
:101A9000AF909F908F907F900C94CE2990910F01E2
:101AA000981738F44CE36FEB70E08FE794E00C94F8
:101AB000CE298093DA010C94570C7F928F929F92DB
:101AC000AF92BF92CF92DF92EF92FF920F931F934C
:101AD000CF93DF93CDB7DEB72C970FB6F894DEBF68
:101AE0000FBECDBF80E090E00E942207823B61F4F0
:101AF00081E090E00E9422078C3A31F482E090E08D
:101B00000E942207823E19F00E940C08EAC08091D0
:101B1000D801863008F4E3C01BEF180F62E771E0CC
:101B20008DEC94E00E94EF34912EE12EF12C85E0B3
:101B3000E80EF11C33E3832E4CE3A42EB12C092DC7
:101B400010E0E016F1060CF482C08091D8018911F2
:101B500003C060E771E002C06EE671E08DEC94E0D6
:101B60000E94BF34F801EE0FFF1FE855FE4F65914C
:101B70007491CE0101960E94953ABE016F5F7F4F2E
:101B80008DEC94E00E94E2348092D6046801CC0C83
:101B9000DD1CCC0CDD1CC60107960E942207082F15
:101BA000C60108960E94220710E0102F0027080F98
:101BB000111D0115110509F442C0C801B5010E94AB
:101BC000C938762E89E0861730F06CE671E08DEC2E
:101BD00094E00E94BF344AE050E0672D8DEC94E021
:101BE0000E94C1356AE671E08DEC94E00E94BF343A
:101BF000C801B5010E94C9388C018A30910530F4C2
:101C000068E671E08DEC94E00E94BF344AE050E059
:101C1000602F8DEC94E00E94C13566E671E08DEC9A
:101C200094E00E94BF34C60106960E9422074AE053
:101C300050E0682F8DEC94E00E94C83506C06DE539
:101C400071E08DEC94E00E94EF34939478CF68E4D7
:101C500071E08DEC94E00E94EF3466E089E894E056
:101C60000E943C24882319F081E08093DC0163E02A
:101C700089E894E00E943C24882371F04091D801C7
:101C8000242F30E080910E0190E00197281739074A
:101C90001CF44F5F4093D80161E089E894E00E9412
:101CA0003C24882339F08091D801882319F0815091
:101CB0008093D80148E265E089E894E00E944E24D0
:101CC00081110E940C0864E089E894E00E943C24A1
:101CD000882339F08091D8010E944E0D02C010E097
:101CE0001DCF2C960FB6F894DEBF0FBECDBFDF918F
:101CF000CF911F910F91FF90EF90DF90CF90BF9009
:101D0000AF909F908F907F9008952F923F924F9227
:101D10005F926F927F928F929F92AF92BF92CF927B
:101D2000DF92EF92FF920F931F93CF93DF93CDB784
:101D3000DEB72E970FB6F894DEBF0FBECDBFE09191
:101D4000DA01F0E0EE0FFF1FE855FE4F6591749148
:101D5000CE0101960E94953A8091DF01843030F4E3
:101D60006DEA70E08DEC94E00E94EF3460EA70E080
:101D70008DEC94E00E94EF344AE050E06091DF0186
:101D80008DEC94E00E94C13568E970E08DEC94E040
:101D90000E94EF346EE870E08DEC94E00E94BF3456
:101DA000BE016F5F7F4F8DEC94E00E94013566E8C5
:101DB00070E08DEC94E00E94BF3489E291E09E8750
:101DC0008D87C12CD12C76016091F0047091F104C3
:101DD0008091F2049091F3046C0D7D1D8E1D9F1D6A
:101DE0000E9439372B013C0120E030E040EA51E409
:101DF0000E94A5360E94A2364B015C0120E030E033
:101E000040EF51E4C301B2010E94A5360E9463383D
:101E10001B012C01ED85FE8512910291FE87ED8755
:101E200020E030E040EE50E4C501B4010E940038EB
:101E300020E030E040E051E40E943E360E940D3741
:101E4000762E20E030E040E851E4C501B4010E9464
:101E500000389B01AC0160E070E080E891E40E94F2
:101E60003D360E940D37B62E20E030E048E052E4C7
:101E7000C201B1010E94003820E030E048E052E4A5
:101E80000E943E360E940D37862F20E0472D6B2D95
:101E90000E94A509F8E0CF0ED11CE11CF11C80E4E2
:101EA000C816D104E104F10409F08ECF64E089E89A
:101EB00094E00E943C24882331F08091D9018093E2
:101EC000DA010E944E0D2E960FB6F894DEBF0FBEBB
:101ED000CDBFDF91CF911F910F91FF90EF90DF90D9
:101EE000CF90BF90AF909F908F907F906F905F90BA
:101EF0004F903F902F9008952F923F924F925F9274
:101F00006F927F928F929F92AF92BF92CF92DF9209
:101F1000EF92FF920F931F93CF93DF93CDB7DEB76E
:101F20002A970FB6F894DEBF0FBECDBF2091EA010D
:101F30003091EB013B832A83265431093D832C8366
:101F400060900A0170900B01C901B3010E94C93869
:101F50006C013091DC013E8320900C0130900D012A
:101F600084E1280E311CEDEFF1E0FA87E98704E007
:101F700012E0E12CF12CFBE0F98396012A5B3F4F44
:101F800038872F8366E0562E4E2C3E81313049F53E
:101F9000E985FA8520813181C1018E0D9F1D2817A9
:101FA0003907F8F4F801608170E080E090E00E9469
:101FB0003B374B015C0120E030E040EC51E4E98527
:101FC000FA8563817481858196810E9400389B0126
:101FD000AC01C501B4010E943E360E940D37F801E4
:101FE0006083F8018081893180F068E10E94BD380A
:101FF000E985FA8520813181280F311D31832083C5
:10200000F80180810E94BD389083E985FA85A0801F
:10201000B1802C813D81A216B30618F4398131506C
:102020003983C501B3010E94C938EF81F8858E1745
:102030009F0708F040C0C816D906E8F58C199D091D
:10204000589EF001599EF00D1124E952FD4F8081F8
:10205000992787FD909597FF03C0919581959109E8
:10206000BC01882777FD8095982F0E943B3720E0A0
:1020700030E040EE50E40E94A5369B01AC0160E0E8
:1020800070E080E090E40E943D36E985FA85638344
:10209000748385839683C501B3010E94C9388C1966
:1020A0009D09589EF001599EF00D1124E952FD4FF3
:1020B000439445822EC0642D70E080E090E00E9441
:1020C000393720E030E040E251E40E94A5369B0120
:1020D000AC0160E070E080E090E40E943D36E9856C
:1020E000FA856383748385839683F8ECAF0EB11C05
:1020F0002A813B81A216B30660F420E030E040E87C
:102100005FE30E943E36E985FA85638374838583A5
:102110009683FFEFEF1AFF0A29853A85265F3F4F26
:102120003A872987065F1F4F3AE0E316F10409F06A
:102130002BCF89818093DF012A960FB6F894DEBFFA
:102140000FBECDBFDF91CF911F910F91FF90EF9008
:10215000DF90CF90BF90AF909F908F907F906F90C7
:102160005F904F903F902F9008957F928F929F9213
:10217000AF92BF92CF92DF92EF92FF920F931F9395
:10218000CF93DF9300910A0110910B018091EA0136
:102190009091EB0186549109B8010E94C9387C01E5
:1021A000C090EC01D090ED014091120170901101AE
:1021B000CFEFD1E0FE01329780819181B8010E947A
:1021C000C938E816F90680F59701240F311D8217EA
:1021D000930750F588819601280F311D87FD3A95A8
:1021E000C9010E964D9700F589809A80AB80BC801E
:1021F00020E030E040EA51E4C501B4010E9400381B
:102200000E940D37762E20E030E040EA50E4C50110
:10221000B4010E94003820E030E040EC50E40E941D
:10222000A5360E940D37462F2A9632E0C336D307D3
:1022300009F0C0CF4093120170921101DF91CF914C
:102240001F910F91FF90EF90DF90CF90BF90AF90D4
:102250009F908F907F9008951092D0041092CF0499
:1022600085EB91E09093CE048093CD0480E196E0DD
:1022700090937E0480937D0408951F93CF93DF9302
:102280001F92CDB7DEB7162FBC0180E595E04983DC
:102290000E94B720612F80E595E00E94642049816B
:1022A000642F80E595E00E94642080E595E00F9022
:1022B000DF91CF911F910C94302140E06DE283E5D6
:1022C00090E00E943D1140E16DE283E590E00E94C4
:1022D0003D114BE061E383E590E00E943D1148E051
:1022E0006DE283E590E00E943D1146E06CE283E5FB
:1022F00090E00E943D1140E86EE283E590E00E948C
:102300003D1164E670E080E090E00E94CF3240E052
:102310006EE183E590E00E943D1140E06FE183E5CE
:1023200090E00E943D1140E060E283E590E00C9473
:102330003D118FE794E00E94042F60EA71E08FE77F
:1023400094E00E94872E1092970480E595E00E9409
:10235000A3200E94FC078091D70181110E945D118A
:1023600060E070E0CB010E947E070E9430080C9470
:10237000570C109211011092EB011092EA010C948B
:1023800099118091D701811104C044E060E172E0AD
:1023900003C045E066E072E08FE794E00E94B22B54
:1023A000823079F02CF4882341F0813041F0089597
:1023B000833059F0843059F0089581E009C00C94BD
:1023C000570C1092D80185E003C00C94B91186E037
:1023D0008093DC010895EF92FF920F931F93CF93A8
:1023E000DF9300D000D0CDB7DEB77C01162FBC0143
:1023F00080E595E02B833C8349835A830E94B72074
:10240000612F80E595E00E94642080E595E00E94C0
:102410003021B70180E595E00E94B72049815A81BB
:10242000B70180E595E00E942D212B81022F3C8190
:10243000132F80E595E00E940C20892B41F080E568
:1024400095E00E941420F80181938F01F2CF80E57E
:1024500095E00F900F900F900F90DF91CF911F910B
:102460000F91FF90EF900C9430210F931F93CF9317
:10247000DF9300D000D000D0CDB7DEB78C019E0135
:102480002F5F3F4F46E050E062E383E590E00E941B
:10249000EB118A8190E0982F88272981822BF801FF
:1024A000918380838C8190E0982F88272B81822BC9
:1024B000938382838E8190E0982F88272D81822BB1
:1024C0009583848326960FB6F894DEBF0FBECDBFEA
:1024D000DF91CF911F910F910895CF93DF9300D09B
:1024E00000D000D0CDB7DEB764E371E08DEC94E0AE
:1024F0000E94EF346FE171E08DEC94E00E94EF34C4
:1025000068E071E08DEC94E00E94EF3466EF70E0DB
:102510008DEC94E00E94EF34CE0101960E943512BA
:1025200066E089E894E00E943C24882319F081E069
:102530008093DC0160E089E894E00E943C248823D9
:1025400031F08B819C819093D6018093D50162E01C
:1025500089E894E00E943C24882331F08B819C819F
:102560009093D4018093D30141E02091D501309123
:10257000D6018091D3019091D401821793070CF07A
:1025800040E04093D20168EE70E08DEC94E00E9450
:10259000BF344091D2012B813C818091D301909135
:1025A000D401442331F0821B930B1816190634F022
:1025B0000BC0281B390B1216130634F462EE70E0C0
:1025C0008DEC94E00E94BF344091D2012B813C817C
:1025D0008091D5019091D601442321F0821B930B69
:1025E000892F03C0281B390B832F881F8827881F3A
:1025F00031F06DED70E08DEC94E00E94BF342696D2
:102600000FB6F894DEBF0FBECDBFDF91CF91089516
:102610002F923F924F925F926F927F928F929F92F2
:10262000AF92BF92CF92DF92EF92FF920F931F93E0
:10263000CF93DF93CDB7DEB729970FB6F894DEBFFF
:102640000FBECDBF4091DD015091DE014F5F5F4F66
:102650005093DE014093DD0180910C0190910D01BA
:102660008A5B9F4F2091EA013091EB01821793071B
:1026700068F48091DC01813049F482E08093DC01D0
:102680006091DF018091DA010E94560841E060E02C
:1026900089E894E00E945C24882321F08091100155
:1026A0008130E1F541E062E089E894E00E945C2439
:1026B000882321F0809110018530A1F541E065E08B
:1026C00089E894E00E945C248823C1F08091110184
:1026D000843020F084508093110102C010921101C7
:1026E00080911001823019F481E080931001809173
:1026F0001001843019F485E08093100141E064E01A
:1027000089E894E00E945C2420911101882371F0F3
:102710008091DC01833009F0BBC308C082E0809364
:102720001001C0CF84E080931001C8CF222319F09C
:1027300021502093110162E089E894E00E94452431
:10274000882329F08091D70181110FC0B0C360E0C8
:1027500089E894E00E9445248111F4CF64E089E87F
:1027600094E00E9445248111EDCF8091D701882308
:1027700009F476C0CE0101960E9435124091D20133
:102780002091D5013091D6018B819C81442319F091
:10279000281B390B04C0BC01621B730B9B01232F48
:1027A000221F2227221F39F020911001213019F019
:1027B00022E0209310012091D3013091D4014423D1
:1027C00031F0281B390B1216130634F00CC0821B93
:1027D000930B181619063CF480911001853019F0FE
:1027E00084E08093100162E089E894E00E9445242F
:1027F000811161C360E089E894E00E944524811161
:102800005AC364E089E894E00E944524811153C3CF
:102810004091D2012091D5013091D6018B819C81CC
:10282000442331F0281B390B1216130644F018C04C
:10283000FC01E21BF30B1E161F0654F011C0209181
:10284000D3013091D401281B390B37FF09C033C3A2
:102850002091D3013091D401821B930B97FD2BC3A0
:10286000809110018230A9F018F4813031F03EC01F
:102870008430D9F0853031F139C02091EC013091AC
:10288000ED012035310594F58091120190E00A9612
:1028900027C02091EC013091ED012035310534F550
:1028A0008091120190E005961BC02091EC013091BF
:1028B000ED01213BFFEF3F07CCF0409112018BEF80
:1028C0009FEF0CC02091EC013091ED01213B4FEFC7
:1028D000340764F04091120186EF9FEF841B910949
:1028E000820F931F9093ED018093EC0166E089E8DD
:1028F00094E00E943C2481111092DC018091EC0153
:102900009091ED012091DA0262EE6203A0011124A0
:10291000841795073CF07EE1279F9001112428172A
:102920003907A4F480911101853118F086958093C0
:10293000110180911101882349F08091E0018130DB
:1029400011F48FEF01C081E08093E00183E6809372
:102950007C0480937B041092F1011092F00110929C
:10296000EF011092EE018091110168E10E94BD38E3
:10297000809312010E94B510F09012012F2D30E0CB
:102980008091EA019091EB01820F931F9093EB01EC
:102990008093EA011092F20160E086E490E0821BED
:1029A000930B76E0462F50E048175907BCF4749F0C
:1029B000D001759FB00D1124A952BD4F420F531F76
:1029C000749FF001759FF00D1124E952FD4F472FC0
:1029D00001900D924A95E1F76F5FE4CF76E4C72E40
:1029E000D12CE6E0EE2EFF20A9F0C6018F19910947
:1029F000E89E8001E99E100D112409521D4F0E948E
:102A0000A707F8012083318342835383648375834E
:102A1000FA94E9CF6091D702709112016703A00187
:102A200011242091EC013091ED01240F351F3093DA
:102A3000ED012093EC018091E101723028F0962F96
:102A400067FD9F5F959501C090E0980F9093E1011D
:102A50008091E001890F0E94650A0E949B0B009102
:102A6000EE011091EF01D0907B04EFEDF2E021E058
:102A700030E058E1E52EF12C65E0C62EDF0111971C
:102A80008C91080F111D87FD1A95C701B9010E948D
:102A9000DD3848E1B42EB60EC09EC001C19E900D37
:102AA0001124B9016C5F7F4F0E94DD38B60EB082F1
:102AB000AB2DBB27A7FDB0954D2D50E0A417B50752
:102AC0000CF4DB2C2F5F3F4F369626343105B1F6E0
:102AD0001093EF010093EE01D0927B048D2D0E94A4
:102AE000160B0E947C0F1092E9011092E80184E518
:102AF00090E09093E7018093E60192EEA92E92E098
:102B0000B92ECC24C394D12C33E0232E312CF501E3
:102B1000339770803196208133978081E090F00167
:102B2000F090F101E80EF11C87FDFA94F092F101AA
:102B3000E092F001FAE2EF0EF11C8091EC0190912D
:102B4000ED01B6010E94DD38E60EF71E3EE1239F3F
:102B5000C0011124B6010E94DD387727C701861B0A
:102B6000970B9093E5018093E4016E0D7F1D7093A8
:102B7000E3016093E20180917C04781608F070C054
:102B800045E0471508F06CC0682E671800E010E0BB
:102B9000862C912CE091E201F091E3012091E40177
:102BA0003091E501061508F051C08091EA0190913D
:102BB000EB018C0D9D1DB1010E94C938CB01B10103
:102BC0000E94C9388F83472D400FE09FC001E19FCD
:102BD000900DF09F900D1124B4010E94DD38E61B8A
:102BE000F70B6091E6017091E701069FC001079F16
:102BF000900D169F900D1124B4010E94DD38E60F50
:102C0000F71F209FC001219F900D309F900D112430
:102C1000B4010E94DD382901461A570A2091E801C3
:102C20003091E901029FC001039F900D129F900D0A
:102C30001124B4010E94DD38CB012F81BF01840D26
:102C4000951D0E94E80B0F5F1F4FA4CF3093E90141
:102C50002093E801F093E701E093E60170927C0491
:102C60008091F201843108F0C8C05FE35C1508F47C
:102C7000C4C0F601E356FC4F149180E1682E611A3E
:102C8000572C5618F501319780818230B1F120F42C
:102C9000813009F445C081C0833009F454C08530C7
:102CA00009F07BC0862D880F5E2D581B862D67FE90
:102CB00002C081E0860D8595581B90E004E0402E0F
:102CC0004701810E911C711A1E141F048CF464E5D7
:102CD000861691046CF401E020E634E0472D692F5C
:102CE000650F812F598798870E94410C98855985D7
:102CF0004A94960D4110E8CF50C06091E201709166
:102D0000E301CB01810F911D843591050CF045C085
:102D1000161617060CF041C001E026EC34E039C06D
:102D20006091E4017091E501862D992787FD9095CA
:102D30008617970794F5643571057CF5661901E0EF
:102D400024EA34E026C06091E4017091E501862D0B
:102D5000992787FD9095861797075CF46435710570
:102D600044F4661901E022E834E0452D812F0E94E9
:102D7000410C6091E2017091E301CB01810F911D43
:102D80008435910554F4161617063CF401E022E848
:102D900034E0452D812F0E94410CF501808188236C
:102DA00061F19091F201943140F51E141F041CF55D
:102DB0009701210F311D24353105ECF490E0019786
:102DC0002AE0289FF001299FF00D1124E550FE4FC5
:102DD000208131818481992787FD9095B6010E94D9
:102DE000DD386E0D67FC63946594661900E0452D2F
:102DF000812F0E94410CF5011082FFEFCF1ADF0AEC
:102E000026E0A20EB11C36E4C316D10409F07FCE31
:102E10000E94790B609110018091E0010E94B10A3B
:102E2000609111016F7120E041E084EA94E00E941A
:102E300002308091DC01833009F041C08091DB01D8
:102E400081508093DB01811104C081E08093DC011B
:102E500036C064E10E94BD38392F3695E82FF0E086
:102E6000EE0FFF1FED5EFE4F0081118164E0630FE6
:102E700021E0492F82E2830F0E94A5098091DD01A4
:102E80009091DE0101979093DE018093DD0117C0E0
:102E9000263908F050CC86E191E0821B9109880F19
:102EA000892F881F990B820F8093110144CC83E0F6
:102EB000809310015ACC83E080931001D1CC2996E5
:102EC0000FB6F894DEBF0FBECDBFDF91CF911F913B
:102ED0000F91FF90EF90DF90CF90BF90AF909F90B9
:102EE0008F907F906F905F904F903F902F900895BC
:102EF0008FE794E00E94F82A8823D9F08091DC01C2
:102F0000823069F028F4882361F0813061F00895FF
:102F1000853059F0863059F0833059F404C00C9450
:102F2000850E0C94C1110C9408130C945D0D0C9437
:102F30006D120895E0910E05F0910F050995E0914D
:102F40001205F09113050994FF920F931F93CF93ED
:102F5000DF93C82FD42F152F062FF72E87FF0AC017
:102F600040E050E0BA0187E70E94A417823008F0E1
:102F70004DC0CF77E0910E05F0910F050995E091D6
:102F80001005F09111050995E0911205F0911305D6
:102F90000995E0911205F091130509958F3FC9F746
:102FA000E0911405F09115058C2F0995E091140519
:102FB000F09115058F2D0995E0911405F0911505F7
:102FC000802F0995E0911405F0911505812F099541
:102FD000E0911405F09115058D2F0995C03421F06D
:102FE000C83421F081E003C085E901C087E8E091A1
:102FF0001405F09115050995CAE0E0911205F091CC
:103000001305099587FF02C0C150B9F7DF91CF9131
:103010001F910F91FF9008959093150580931405CB
:10302000709313056093120550931105409310059A
:1030300030930F0520930E050895EF92FF920F93A2
:103040001F93CF93DF9300D000D01F92CDB7DEB790
:1030500014E6E0911205F091130509951150C9F796
:1030600040E050E0BA0180E40E94A417813009F0EA
:1030700057C04AEA51E060E070E088E40E94A4177B
:10308000813039F57E0185E0E80EF11C8E010F5F7D
:103090001F4FE0911205F09113050995F8018193F6
:1030A0008F01EE15FF05A9F78B818130C9F58C8161
:1030B0008A3AB1F508EA11E640E050E060E070E4D9
:1030C00089EE0E94A4178823A9F101501109A1F7E4
:1030D00027C040E050E0BA0189EE0E94A417823078
:1030E00020F492E0F92E99EE03C0FF24F39491E4CA
:1030F00008EA11E640E050E0BA01892F9D830E9462
:10310000A4179D81882321F00150110999F708C067
:1031100040E052E060E070E080E50E94A417811179
:10312000F12CF0921F080E949A1781E0FF2009F10C
:1031300080E01FC040E050E0BA018AE70E94A41777
:103140008111EECF8E010F5F1F4FE0911205F091BC
:1031500013050995F80181938F01EE15FF05A9F775
:10316000898186FF03C02CE0F22EDBCF84E0F82EAD
:10317000D8CF0F900F900F900F900F90DF91CF91BD
:103180001F910F91FF90EF9008958F929F92AF92B1
:10319000BF92CF92DF92EF92FF920F931F93CF9344
:1031A000DF931F92CDB7DEB76C0179014801E89437
:1031B00097F88114910409F484C0C401820F931F0D
:1031C0008130924008F07DC080911F0883FD07C0C8
:1031D000E9E0440F551F661F771FEA95D1F781E597
:1031E0000E94A417811165C048EEA42E43E0B42EBE
:1031F000E0911205F091130509958F3F29F481E0C4
:10320000A81AB108A9F755C08E3F09F052C032E0A4
:10321000A32EBA2CAE18BF08A818B908E114F104FF
:1032200049F0E0911205F0911305099591E0E91A32
:10323000F108F4CF17FF28C0E0910805F0910905C7
:103240000995E0910C05F0910D050995E0911205A5
:10325000F09113050995F6010995E0910A05F091A1
:103260000B0589830995F1E08F1A910889818114F2
:10327000910411F08111E5CFE0910605F091070569
:103280000995A80CB91C0CC0E0911205F09113052A
:103290000995D6018D936D01B1E08B1A9108A1F7C4
:1032A000E0911205F09113050995E1E0AE1AB1081D
:1032B000B9F70E949A1781E090E0892821F480E014
:1032C00002C084E090E00F90DF91CF911F910F91A9
:1032D000FF90EF90DF90CF90BF90AF909F908F9036
:1032E00008950F931F93E0911605F09117059C0127
:1032F0002250310940855185425051092417350724
:1033000068F4A181B0E00E943239028913892489CE
:103310003589600F711F821F931F03C060E070E04A
:10332000CB011F910F910895CF93DF93EC01E091B2
:103330001605F0911705198218828C819D818130C4
:103340009105B9F0208531858217930790F49F830A
:103350008E83009719F00E94711904C066857785E5
:1033600080899189688779878A879B8780E090E048
:1033700002C081E090E0DF91CF9108958F929F92FB
:10338000AF92BF92CF92DF92EF92FF920F931F9373
:10339000CF93DF9300D000D0CDB7DEB77C01C090D3
:1033A0001605D09017058230910508F473C0F60118
:1033B00080859185E816F90608F06CC0808181301F
:1033C00021F0823009F44CC065C04701969487947F
:1033D0008E0C9F1C94013170892C99248694A12C09
:1033E000B12CF60182859385A485B585B501A4012C
:1033F000480F591F6A1F7B1F2F3FF1E03F0729F03D
:1034000002E010E0CE0101961BC001E010E02FEFBA
:1034100031E0CE0101960E94C518892BD9F5F6013D
:1034200042855385648575854F5F5F4F6F4F7F4F32
:10343000480D591D6A1D7B1D20E030E0CE0102962B
:103440000E94C518892B31F589819A81E0FE06C05A
:1034500024E0969587952A95E1F71EC09F701CC0C1
:1034600097013327220F331FEF2CFF24F6014285EB
:103470005385648575854E0D5F1D611D711D02E0CC
:1034800010E0CE0101960E94C518892B19F489819C
:103490009A8102C081E090E00F900F900F900F9002
:1034A000DF91CF911F910F91FF90EF90DF90CF9020
:1034B000BF90AF909F908F900895EF92FF920F93DF
:1034C0001F93CF93DF93EC01E0901605F090170562
:1034D000088119810F5F1F4F19F483E090E049C004
:1034E000488559856A857B854115510561057105BA
:1034F000A1F3C8018F709927892BA1F54F5F5F4F0A
:103500006F4F7F4F488759876A877B878E819F815E
:10351000F701009731F48481958108171907E8F6BF
:1035200021C0218130E021503109A80164E0569585
:1035300047956A95E1F724233523232B99F40E94BC
:10354000BE198230910598F0F701208531858217E8
:10355000930718F69F838E830E9471196887798775
:103560008A879B871983088380E090E002C081E00E
:1035700090E0DF91CF911F910F91FF90EF90089510
:10358000CF92DF92EF92FF920F931F93CF93DF932F
:10359000EC016A017B0102E010E02EEF31E00E94B5
:1035A000C518892BC1F48881998185359A4AA9F477
:1035B00026E330E0B701A601CE010E94C518892B91
:1035C00041F481E0288139812634314439F480E0A6
:1035D00005C081E003C083E001C082E0DF91CF91AC
:1035E0001F910F91FF90EF90DF90CF900895BF92C1
:1035F000CF92DF92EF92FF920F931F93CF93DF93BF
:10360000EC016B01FB0180818F3219F4FFEFCF1ABF
:10361000DF0A1D821C82F6018081803260F4CE01B7
:103620000E949419E0911605F09117050680F78124
:10363000E02D1082B0C0E0E2BE2EEA81FB81DF0106
:10364000CF010B96A817B90711F0BD92FBCF50E040
:1036500080E068E071E0780FD601A80FB11D4C91B1
:103660004032D0F04F32C1F04E3209F47AC05617D2
:1036700008F068C04F3708F065C0842F90E0AFE8CD
:10368000B1E02D91222309F460C0332727FD309546
:1036900028173907B1F756C0552309F453C0C70E90
:1036A000D11C81E0403208F080E08387CE010E9487
:1036B00094190097B1F5E0911605F0911705E68091
:1036C000F780288139812F70332775E0220F331F4F
:1036D0007A95E1F7488559856A857B8500E210E097
:1036E000C7010E94C518892B39F5F701808188230D
:1036F000D9F0838583FD10C06A817B81C701DB011E
:103700009B01255F3F4FA217B30781F1FC01519147
:10371000CF014D915417B9F3CE010E945D1A009765
:1037200081F283309105B9F5EA81FB818385882395
:1037300031F083E090E02FC081E090E02CC084E085
:1037400090E029C085E090E026C08FE9840F8A319F
:1037500008F44052DF01A50FB11D4C935F5F872F26
:1037600079CF683079F758E06BE0F9CFFB018385BA
:1037700081110FC0E0911605F09117050680F781C1
:10378000E02D838584FFDBCF828D938D9D838C8399
:1037900054CF80E090E0DF91CF911F910F91FF9087
:1037A000EF90DF90CF90BF9008954F925F926F920D
:1037B0007F92AF92BF92CF92DF92EF92FF920F93E0
:1037C0001F93CF93DF93CDB7DEB7A8970FB6F894CA
:1037D000DEBF0FBECDBF5C0110921705109216051B
:1037E000009709F4D0C00E941D1880FDCFC040E0B2
:1037F00050E0BA01CE0101960E94C01A813009F54D
:1038000000E110E02EEB31E040E050E0BA01CE01E3
:1038100001960E94C518892B19F081E090E0B8C08C
:103820008D81811103C089E090E0B2C049845A843F
:103830006B847C84B301A201CE0101960E94C01A60
:1038400003C0412C512C3201833039F38111EBCF6D
:1038500004E210E02DE030E0B301A201CE010196B8
:103860000E94C518892BC9F62A853B8540E050E0A7
:10387000211531054105510521F4288D398D4A8DD9
:103880005B8DAC81B0E00E9441396DA37EA38FA314
:1038900098A70A811B8120E030E0400E511E621E75
:1038A000731ED5011A964D925D926D927C921D9772
:1038B000498111964C931197CD80DE801596DC924C
:1038C000CE9214978F819885A0E0B0E00097A10573
:1038D000B10521F48C899D89AE89BF89F4E0D69425
:1038E000C794FA95E1F7E12CF12CBC01CD01601BE6
:1038F000710B820B930B0DA11EA12FA138A5601B8C
:10390000710B820B930B6C197D098E099F09242F73
:1039100030E040E050E00E94F1382E5F3F4F4F4FC3
:103920005F4FD50119963C932E931897273FBFE020
:103930003B074105510540F0273F3F4F41055105E9
:1039400008F071CF82E001C081E0D5018C930DA118
:103950001EA12FA138A5400E511E621E731E1E9679
:103960004D925D926D927C9251974C0C5D1C6E1C39
:103970007F1CF501428A538A648A758A1282B0924A
:103980001705A092160580E090E002C082E090E06A
:10399000A8960FB6F894DEBF0FBECDBFDF91CF91D2
:1039A0001F910F91FF90EF90DF90CF90BF90AF905D
:1039B0007F906F905F904F9008950F931F93CF93D8
:1039C000DF93CDB7DEB7E8970FB6F894DEBF0FBE32
:1039D000CDBF00911605109117050115110569F16C
:1039E000F80112829E012F5F3F4F37832683205EAE
:1039F0003F4F38AB2FA7BC01CE018D960E94F71A1E
:103A00000097F9F489818823D1F08C8584FD17C053
:103A10008B8D9C8DF801978F868F8D8D9E8DAF8DB0
:103A2000B8A1828F938FA48FB58F168A178A108EB4
:103A3000118E81E0828380E003C088E001C083E0D2
:103A400090E0E8960FB6F894DEBF0FBECDBFDF91D1
:103A5000CF911F910F9108952F923F924F925F92B5
:103A60006F927F928F929F92AF92BF92CF92DF928E
:103A7000EF92FF920F931F93CF93DF9300D000D06C
:103A8000CDB7DEB789839A837B014A018091160501
:103A9000909117059C838B83FA0111821082009705
:103AA00009F4BBC0FC01828180FFBAC0828D938D76
:103AB000A48DB58D46895789608D718D841B950BBA
:103AC000A60BB70BA70160E070E084179507A60767
:103AD000B70708F47C01A980BA80612CB2E07B2E84
:103AE000E114F10409F496C0EB81FC812688378843
:103AF000408C518CD201C1019170AA27BB27892B20
:103B00008A2B8B2B09F044C0218130E040E050E04B
:103B1000C201B101A9E09695879577956795AA9519
:103B2000D1F70E94F138672B682B692BA9F4EB8140
:103B3000FC8123282428252819F4868D978D04C01C
:103B400080A191A10E94BE19EB81FC818230910578
:103B500080F091A380A31382EB81FC8180A191A1CD
:103B60000E947119EB81FC81611571058105910538
:103B700011F4128258C02381DC01CB01820F911D08
:103B8000A11DB11D82A393A3A4A3B5A32F5F23837B
:103B9000EB81FC81268937893170C301821B930B2D
:103BA00067018E159F0508F46C01EB81FC81828111
:103BB00042A153A164A175A1860186FF04C01068CB
:103BC00089819A8101C0C5010E94C518009741F002
:103BD000EB81FC811282029731F586E090E025C0EE
:103BE000AC0CBD1CEB81FC8186899789A08DB18DC1
:103BF0008C0D9D1DA11DB11D868B978BA08FB18F44
:103C0000F401808191818C0D9D1D91838083EC183E
:103C1000FD0866CF80E090E008C088E090E005C035
:103C200087E090E002C081E090E00F900F900F904D
:103C30000F90DF91CF911F910F91FF90EF90DF9048
:103C4000CF90BF90AF909F908F907F906F905F903C
:103C50004F903F902F9008954F925F926F927F9276
:103C60008F929F92AF92BF92CF92DF92EF92FF928C
:103C70000F931F93CF93DF9300D000D0CDB7DEB763
:103C80009B0100911605109117050115110509F406
:103C9000D0C0D80112964C91129740FFCDC05A96D1
:103CA0004D915D916D917C915D9769017C014C1501
:103CB0005D056E057F0510F46A017B01F8014688F9
:103CC0005788608C718C168A178A108E118EC114D9
:103CD000D104E104F10409F4B2C08180912CA12C3B
:103CE000B12C39E0880C991CAA1CBB1C3A95D1F761
:103CF0004114510461047104C9F1B1E04B1A510837
:103D000061087108C701B601615071098109910903
:103D1000A50194010E94F13829833A834B835C8387
:103D2000C301B201A50194010E94F13889819A81F1
:103D3000AB81BC8182179307A407B507B8F0882729
:103D40009927DC0188199909AA09BB0984219521C1
:103D5000A621B721F801868B978BA08FB18FC81A47
:103D6000D90AEA0AFB0A80A191A128C0D8015E966F
:103D70008D919C915F9791969C938E9390971EC086
:103D80000E94BE1982309105F8F0F8012085318536
:103D900082179307C8F4F80191A380A34689578935
:103DA000608D718D480D591D6A1D7B1D468B578B8B
:103DB000608F718FC818D908EA08FB088C149D041D
:103DC000AE04BF04E8F204C0D80112961C921FC0D2
:103DD000F80146895789608D718D4C0D5D1D6E1DF2
:103DE0007F1D468B578B608F718F29E0F694E79487
:103DF000D794C7942A95D1F7C394C3820E947119AE
:103E0000611571058105910529F4F801128281E09F
:103E100090E017C0DC01CB010197A109B1098C0D1D
:103E2000911DA11DB11DF80182A393A3A4A3B5A365
:103E300006C088E090E005C087E090E002C080E026
:103E400090E00F900F900F900F90DF91CF911F9106
:103E50000F91FF90EF90DF90CF90BF90AF909F9029
:103E60008F907F906F905F904F9008950F931F9366
:103E7000CF93DF93CDB7DEB7AC970FB6F894DEBF24
